:100000000C946C020C94B3020C94B3020C94B302E3
:100010000C94B3020C94B3020C94B3020C94B3028C
:100020000C94B3020C94B3020C94581C0C942B1D2A
:100030000C94CC130C94B3020C94B3020C94B30242
:100040000C94B3020C94B3020C94B3020C94B3025C
:100050000C94B3020C9434140C94B3020C94B302B9
:100060000C94B3020C94B3020C94B3020C94B3023C
:100070000C94B3020C94B3020C94B3020C94B3022C
:100080000C94B3020C94B3020C94B3020C94B3021C
:100090000C94B3020C94B3020C94B3020C94B3020C
:1000A0000C94B3020C94B3020C94B30229003A00EE
:1000B0003B002A002B002F003000310039003400B3
:1000C00028000000E1000000E5000000E000E3007F
:1000D000E200E40001000100010001000100010054
:1000E000010001000100010001000000010000000A
:1000F00001000000010001000100010001000100F9
:1001000001000100010001000100010001000100E7
:1001100001000000010000000100000001000100DA
:1001200001000100010001000100010001000100C7
:1001300001000100010001000100000001000000B9
:1001400001000000010001000100010001000100A8
:100150000100010001000100010001000100010097
:10016000010000000100000001000000010001008A
:100170000100010001000100010001000100010077
:100180000100010001000100010000000100000069
:100190000100000001000100010001000100010058
:1001A0000100010001000100010001000100010047
:1001B000010000000100000001000000010001003A
:1001C0000100010001000100010001000100010027
:1001D0000100010001000100010000000100000019
:1001E0000100000001000100010001000100010008
:1001F00001000100010001000100010001000100F7
:1002000001000000010000000100000001000100E9
:1002100001000100010001000100010001000100D6
:1002200001000100010001000100000001000000C8
:1002300001000000010001000100010001000100B7
:1002400001000100010001000100010001000100A6
:100250000100000001000000010000000100010099
:100260000100010001000100010001000100010086
:100270000100010001000100010000000100000078
:100280000100000001000100010001000100010067
:100290000100010001000100010001000100010056
:1002A0000100000001000000010000000100010049
:1002B0000100010001000100010001000100010036
:1002C0000100010001000100010000000100000028
:1002D0000100000001000100010001000100010017
:1002E0000100010001000100010001000100010006
:1002F00001000000010000000100000001000100F9
:1003000001000100010001000100010001000100E5
:1003100001000100010001000100000001000000D7
:1003200001000000010001000100010012036B0048
:100330006500790062006F006100720064000000D7
:10034000160371006D006B006200750069006C009F
:1003500064006500720000000403090409026D00D6
:10036000040100A0FA0904000001030101000921B1
:10037000110100012240000705810308000A090459
:1003800001000103010200092111010001224D00B9
:100390000705820308000A090402000103000000A7
:1003A0000921110100012236000705830308000A14
:1003B00009040300010300000009211101000122CA
:1003C000390007058403200001120110010000001C
:1003D00008EDFE606001000102000105010906A1AF
:1003E00001050719E029E715002501950875018128
:1003F00002050819012905950575019102950175F8
:100400000391010507190029F71500250195F875D5
:10041000018102C005010980A101850216010026A3
:1004200003001A81002A8300751095018100C00520
:100430000C0901A1018503160100269C021A010086
:100440002A9C02751095018100C005010902A101D5
:100450000901A100050919012905150025019505C6
:10046000750181029501750381010501093009318A
:100470001581257F95027508810609381581257F2C
:10048000950175088106050C0A38021581257F95AE
:100490000175088106C0C005010906A101050719FB
:1004A000E029E71500250195087501810295017580
:1004B0000881010508190129059505750191029525
:1004C00001750391010507190029FF150026FF009A
:1004D000950675088100C00011241FBECFEFDAE039
:1004E000DEBFCDBF04B603FE27C0809110029091FD
:1004F0001102A0911202B09113028730904BA740D5
:10050000B04BD1F41092100210921102109212020C
:100510001092130214BE84B7877F84BF0FB6F8947D
:10052000A8958091600088618093600010926000BF
:100530000FBEE0E0F8E3099511E0A0E0B1E0EEEDD8
:10054000F0E402C005900D92A033B107D9F722E084
:10055000A0E3B1E001C01D92A031B207E1F70E9413
:10056000A7190C946D200C94000090E080E0089591
:100570000895089581E00895089581E008950C9408
:10058000BA020E94480C2FEF84E39CE02150804087
:100590009040E1F700C000000C945914FF920F93B3
:1005A0001F93CF93DF938C01FC01C081D181809197
:1005B0005B0181113FC082818823B9F1CE010E9485
:1005C000AD11F82E682FCE010E945511BE018F2D5E
:1005D0000E941504EC01B8010E94BF02882309F4AF
:1005E0004AC0B801CE010E942506882309F443C001
:1005F000C531F0E7DF0718F5C23080E7D80708F00B
:100600004BC0C115E0E7DE0789F1C130D047D1F119
:1006100081E08093320180933301C801DF91CF9153
:100620001F910F91FF900C94BD02CE010E94831187
:10063000F82ECCCFCE010E94AD11BE01C9CFCC3374
:1006400080E7D80709F4ACC0CD33D04709F7F801EB
:100650008281882309F4CBC0109233010E94FE13DB
:10066000909331018093300180E2A7C0F80182812C
:1006700081110E94C10280E0DF91CF911F910F9103
:10068000FF900895F80182818823A9F38091D00119
:1006900081608093D001EFCFF8018281882309F433
:1006A000BCCF0E945E13811102C00E9444130E94BD
:1006B0007B1390E09093020280930102FE01E350CD
:1006C000F047809101028160E231F105C8F4E559FB
:1006D000FC4F0C941D207D0389038D03910395032A
:1006E00099039D03A103A503A903AD03B103B503BA
:1006F000B903BD03C103C503C90380910102826030
:1007000080930102809101020E947F130E94480C95
:10071000B2CF809101028460F3CF809101028860A2
:10072000EFCF809101028061EBCF80910102806266
:10073000E7CF809101028064E3CF8091010280685D
:10074000DFCF809101028460EACF809101028E7F29
:10075000D7CF809101028D7FD3CF809101028B7F13
:10076000CFCF80910102877FCBCF809101028F7E16
:10077000C7CF809101028F7DC3CF809101028F7B13
:10078000BFCF809101028F77BBCF809101028B7F19
:10079000EACF90910102892F97FB87F98058B0CF5B
:1007A000F8018281882361F0109232010E94FE13C9
:1007B000909331018093300182E00E94D2095BCF97
:1007C0008091320181110FC08091300190913101EF
:1007D0000E940A14883C910530F486E20E94A70822
:1007E00086E20E94830982E00E94D90944CF809169
:1007F000330181110FC080913001909131010E942D
:100800000A14883C910530F487E20E94A70887E229
:100810000E94830980E2E8CF0C9474060C9476065B
:100820000C94BC020C9410040895E72FF0E095E0BE
:10083000899FE00DF11D1124EE0FFF1FEE0FFF1F2A
:10084000E60FF11DEE0FFF1FE455FF4F85919491C8
:100850000895FC01EE0FFF1FE45DFC4F859194911C
:1008600008950E9415040E94A405811520E49207B2
:1008700008F08DC0811540E3940708F0E8C0803E81
:10088000910508F071C0803C910508F0CCC0883A11
:10089000910580F4853A910508F0CAC08130910530
:1008A00009F46EC020F08430910508F069C090E032
:1008B00080E008958D3B9105D0F7883A910509F4C1
:1008C00004C1893A910509F403C18A3A910509F4F2
:1008D00002C18B3A910509F401C18C3A910509F4E2
:1008E00000C18B3B910509F4FFC08C3B910509F4D5
:1008F000FEC08D3A910509F4FDC0803B910509F4D5
:10090000FCC08E3A910509F4FBC08F3A910509F4B9
:10091000FAC0813B910509F4F9C0823B910509F4C5
:10092000F8C0833B910509F4F7C0843B910509F4B5
:10093000F6C0853B910509F4F5C0863B910509F4A5
:10094000F4C0873B910509F4F3C0883B910509F495
:10095000F2C0893B910509F4F1C08A3B910509F485
:10096000F0C080E094E408958F3F910509F048F4C9
:10097000803F910508F067C0883E910508F097CF49
:100980000895811520E2920708F05FC0089581154F
:1009900043E5940760F5811522E5920708F062C0EF
:1009A000811541E5940708F058C0811520E59207AC
:1009B00008F450C09C0154E0369527955A95E1F70C
:1009C000922F9370482F437021E030E002C0220F35
:1009D000331F4A95E2F73C68392B869586958370DC
:1009E00040E2849FC0011124822B932B089581152E
:1009F00045E5940750F4811524E5920708F446C0B4
:100A0000982F8827846F906A0895811546E594078A
:100A100008F450C09C0130569F702115304108F0F9
:100A200046CF90620895805C91090E942904089540
:100A3000853A910509F443C0863A910509F042C010
:100A400082E890E40895906508959F70EECF99270D
:100A5000906C08959F70906A0895982F8827816FF1
:100A6000906A0895AC014370552721E030E002C040
:100A7000220F331F4A95E2F78695869540E2849FC0
:100A8000C0011124822B932B9C680895AC01437004
:100A9000552721E030E002C0220F331F4A95E2F7CC
:100AA0008695869540E2849FC0011124822B932B6A
:100AB0009A680895982F882788279F71B2CF81E878
:100AC00090E4089583E890E4089582EE94E4089514
:100AD00089EE94E408958AEE94E4089585EB94E415
:100AE000089586EB94E4089583EB94E4089584EBF1
:100AF00094E4089587EB94E408958CEC94E40895CD
:100B00008DEC94E4089583E895E408958AE895E4EB
:100B1000089582E995E4089584E995E4089581E2D1
:100B200096E4089583E296E4089584E296E40895B5
:100B300085E296E4089586E296E4089587E296E4D5
:100B400008958AE296E41CCF8238910549F1B0F409
:100B50008133910509F45CC048F48932910509F4A8
:100B600052C08A32910509F458C008958533910521
:100B700009F444C08933910599F00895833E9105A5
:100B800031F138F4803E910591F0823E9105B1F04B
:100B90000895863E910511F1873E910541F1089532
:100BA000209101022370C9F080EE90E00895209119
:100BB000010220FF12C089E390E008952091010214
:100BC00022FF0BC024FF2EC090E080E0089520910A
:100BD000010222FD2AC024FDF7CF089520910102D1
:100BE00023FFFBCF24FDF0CF87EE90E00895209106
:100BF000010223FFF0CF86EE90E0089520910102DC
:100C000025FD16C008952091010225FD14C0089508
:100C10002091010226FD12C008952091010226FDB7
:100C200010C0089583EE90E0089582EE90E008955C
:100C300089E290E0089585E390E008958AE290E0EB
:100C4000089581E390E0C9CF08950F931F93CF9348
:100C50008C01FB018281811106C0C1E08C2FCF91F4
:100C60001F910F910895C0914101C11125C0053117
:100C7000104799F70E94240681E0809341010E9469
:100C8000FE139093400180933F0110923401109223
:100C900036011092350110923801109237011092EE
:100CA0003A011092390110923C0110923B011092CE
:100CB0003E0110923D01D2CF80913F0190914001C1
:100CC0000E940A14883C910540F680913401E82F77
:100CD000F0E0EE0FFF1FEB5CFE4F118300838F5F90
:100CE00080933401C0E0BACF0C94B8020C94B902DE
:100CF000CF93DF9385B7806885BF85B7806885BF50
:100D0000A7E1B1E04CE151E0C1E0D0E08D91E82FE6
:100D1000E295EF70F0E061A18F709E0101C0220F9B
:100D20008A95EAF7922F9095962391A382A1822B20
:100D300082A34A175B0751F7A3E1B1E061E070E0DD
:100D40008D91E82FE295EF70F0E041A18F709B014B
:100D500001C0220F8A95EAF7922F9095942391A3D0
:100D600082A1822B82A381E0A731B80749F71092B4
:100D700047011092420110924801109243011092D3
:100D800049011092440110924A01109245011092BB
:100D90004B0110924601DF91CF910C940C046F929D
:100DA0007F929F92AF92BF92CF92DF92EF92FF928B
:100DB0000F931F93CF93DF93C2E4D1E007E111E0DB
:100DC000EE24E394F12CDD24D39478811882D801A9
:100DD0008D918D01E82FE295EF70F0E091A18F7079
:100DE000A70101C0440F8A95EAF7892F842B81A3BC
:100DF00082A1942E9094892182A3B0EABA95F1F74A
:100E000033E1632E31E0732E90E080E0D3013D9119
:100E10003D01A32EA2942FE0A222B12CD5019096E1
:100E2000CC9068813F70D70102C0AA0FBB1F3A95D2
:100E3000E2F79D012C2109F056C02E2D082E01C08D
:100E4000220F0A94EAF7262B288301968430910515
:100E5000E9F681A1892181A382A1842B82A38881C3
:100E6000781741F0D0924C010E94FE1390934E01EE
:100E700080934D012196B1E00C311B0709F0A5CFFD
:100E800080914C018823F1F080914D0190914E01A9
:100E90000E940A140697B0F08091420180934701A6
:100EA00080914301809348018091440180934901DE
:100EB0008091450180934A018091460180934B01C6
:100EC00010924C010E940E0481E0DF91CF911F919E
:100ED0000F91FF90EF90DF90CF90BF90AF909F90D9
:100EE0007F906F90089520E0AECFE82FF0E0E95BAF
:100EF000FE4F80810895089590935401809353018B
:100F00000895E0915301F0915401309721F0019040
:100F1000F081E02D099480E00895E0915301F09173
:100F20005401309721F00280F381E02D0994089557
:100F3000E0915301F0915401309721F00480F58144
:100F4000E02D099408952091510130915201281704
:100F5000390771F09093520180935101E091530150
:100F6000F0915401309721F00680F781E02D09942B
:100F7000089520914F01309150012817390771F0E1
:100F80009093500180934F01E0915301F0915401EF
:100F9000309721F00084F185E02D0994089508959B
:100FA0000C94CF070E94F5130E9478060C94BE148F
:100FB000BF92CF92DF92EF92FF920F931F93CF9346
:100FC000DF93CDB7DEB72A970FB6F894DEBF0FBE1A
:100FD000CDBF0E94CF0686E5C82E81E0D82E10E056
:100FE00000E0B02E802F0E947507E82EF601F190E8
:100FF0006F01F81609F45AC08091D00181FD0E945A
:101000007B0790E080E0FE242F2D30E0482FB901CF
:10101000082E02C0759567950A94E2F760FF41C0FB
:101020008E83BF8281E090E06C0102C0CC0CDD1C9D
:101030004A95E2F72E2D30E02C213D21232B09F497
:1010400080E088870E94FE138160782F9A878987C5
:101050004E815F8168858A850E947D08F801EA5A81
:10106000FE4F80818C2580830E9441170E9481075A
:1010700090915501891789F10E948107809355014C
:101080002A960FB6F894DEBF0FBECDBFDF91CF9189
:101090001F910F91FF90EF90DF90CF90BF900C9435
:1010A000120401968430910509F0B0CF0F5F1F4FF5
:1010B0000530110509F095CF8FEF89838A831B8254
:1010C0000E94FE138160782F9D838C8349815A8111
:1010D0006B818D810E947D08C7CF2A960FB6F89448
:1010E000DEBF0FBECDBFDF91CF911F910F91FF905B
:1010F000EF90DF90CF90BF900895CF93DF93CDB75F
:10110000DEB72B970FB6F894DEBF0FBECDBF4F836F
:10111000588769877A878B871E821D8285E0FE014A
:101120003796DE01119601900D928A95E1F749817B
:101130005A816B817C818D819E812B960FB6F894AC
:10114000DEBF0FBECDBFDF91CF910C94FA0E882386
:1011500009F4D8C0823871F40E94810781FDD2C0A1
:1011600089E30E944D120E94151389E30E948A129E
:101170000C941513833859F40E94810780FDC2C076
:1011800083E50E944D120E94151383E5EFCF84384A
:1011900059F40E94810782FDB5C087E40E944D1278
:1011A0000E94151387E4E2CF9CEF980F913A18F450
:1011B0000E944D12DDCF90E2980F983050F4877066
:1011C00091E001C0990F8A95EAF7892F0E94CC120D
:1011D000CFCF9BE5980F933070F4853A31F0863A83
:1011E00039F083E890E00C94A30781E890E0FBCF0E
:1011F00082E890E0F8CF98E5980F953108F082C02A
:10120000883A09F440C0893A09F440C08A3A09F49E
:1012100040C08B3A09F440C08C3A09F440C08B3B83
:1012200009F440C08C3B09F440C08D3A09F440C039
:10123000803B09F440C08E3A09F440C08F3A09F46B
:1012400040C0813B09F440C0823B09F440C0833B6D
:1012500009F440C0843B09F440C0853B09F440C018
:10126000863B09F440C0873B09F440C0883B09F441
:1012700040C0893B09F440C08A3B09F440C090E07B
:1012800080E00C94B90782EE90E0FBCF89EE90E00D
:10129000F8CF8AEE90E0F5CF85EB90E0F2CF86EBC9
:1012A00090E0EFCF83EB90E0ECCF84EB90E0E9CFE0
:1012B00087EB90E0E6CF8CEC90E0E3CF8DEC90E014
:1012C000E0CF83E891E0DDCF8AE891E0DACF82E9F0
:1012D00091E0D7CF84E991E0D4CF81E292E0D1CF01
:1012E00083E292E0CECF84E292E0CBCF85E292E03F
:1012F000C8CF86E292E0C5CF87E292E0C2CF8AE211
:1013000092E0BFCF0895882309F44BC0823871F46E
:101310000E94810781FF45C089E30E944D120E940F
:10132000151389E30E948A120C941513833859F41B
:101330000E94810780FF35C083E50E944D120E9404
:10134000151383E5EFCF843859F40E94810782FF9B
:1013500028C087E40E944D120E94151387E4E2CF53
:101360009CEF980F913AF0F290E2980F983050F479
:10137000877091E001C0990F8A95EAF7892F0E9442
:10138000D212D2CF9BE5980F933020F490E080E00A
:101390000C94A307885A853120F490E080E00C94E7
:1013A000B9070895882321F00E94CC120C941513DC
:1013B0000895882321F00E94D2120C9415130895E9
:1013C0008F929F92AF92BF92DF92EF92FF920F9314
:1013D0001F93CF93DF937C01D62FC72FFC0105818C
:1013E00002950F70128111110E94EB120E94461299
:1013F000D82E882371F0112321F180E28D0F8830DF
:1014000000F182E00E9430120E94461291E0D82E34
:10141000D926EC2FE295EF70F0E0EF5EF54F0C94DB
:101420001D20230A230A730A730AB50AD10A500A37
:10143000500ADC0A500A740B740BE70B500A500A6E
:10144000F00BD12CE6CF0C2F0F70C07F11F002955E
:10145000007F1123A9F0002359F080E28D0F88301E
:1014600010F0D11109C0802F0E94CC120E941513D8
:101470008D2F0E94A70814C0802F0E94DD12F6CF86
:101480008D2F0E948309002359F080E28D0F883050
:1014900010F0D11124C0802F0E94D2120E94151387
:1014A000DD2009F4A4C10E94231280FDA0C1F70130
:1014B00012820E941D120E949910C7010E94030C03
:1014C0000E941D12DF91CF911F910F91FF90EF901D
:1014D000DF90BF90AF909F908F900C94BA10802FA8
:1014E0000E94E312DBCFFC2FFF70BF2EC07FC03203
:1014F00019F0B29480EFB822DD2369F0D13029F1E0
:10150000112369F1002359F0F701858180FFB0CFE5
:101510008F70858304C0112361F0011104C08B2DED
:101520000E94D209BDCF8B2D0130D1F70E94FF124E
:10153000B7CF011106C00E9402138B2D0E94D9095A
:10154000AFCF013009F4ACCFF6CF112321F0063034
:1015500008F0A6CFE4CF053008F0A2CFEECF0023ED
:1015600061F38D2F0E9483099BCF8C2F86958695E2
:10157000837069F0813009F093CF8D2F9C2F937089
:10158000111102C090E080E00E94B90789CF8D2F31
:101590009C2F9370111102C090E080E00E94A3077D
:1015A0007FCF8D2F112329F00E944A160E943617F3
:1015B00077CF0E94B216FACF8C2F837009F047C004
:1015C00011116ECF2D2F229526952770220F220FF5
:1015D0006D2F6F70862E912CB12CA12C022E04C081
:1015E000880C991CAA1CBB1C0A94D2F760E070E01E
:1015F000CB01D4FF0FC06FE070E080E090E004C04A
:10160000660F771F881F991F2A95D2F760957095EE
:1016100080959095C695C695C370C23051F080F400
:10162000682979298A299B29C13071F00E944210CA
:1016300037CF682979298A299B290E945E1030CFEB
:101640000E944210C501B4010E94261029CF869540
:10165000112311F08C2F8170882309F421CF2D2FB5
:10166000229526952770220F220F6D2F6F70862EE0
:10167000912CB12CA12C022E04C0880C991CAA1C00
:10168000BB1C0A94D2F760E070E0CB01D4FF0FC01E
:101690006FE070E080E090E004C0660F771F881F65
:1016A000991F2A95D2F76095709580959095C6956B
:1016B000C695C370C23051F080F4682979298A290F
:1016C0009B29C13071F00E941C11EACE682979294A
:1016D0008A299B290E943811E3CE0E941C11C50162
:1016E000B4010E940011DCCEE0E2ED0FE53108F01C
:1016F00062C0F0E0E258F44F0C941D20930B930B62
:10170000930B930B930B930B930B930B930B930BE9
:10171000930B930B930B930B930B930BA00BAE0BB1
:10172000B50BBC0BC60BDF708C2F8F71112321F012
:101730000E9499108D2FF4CE0E94BA108D2FFECEEC
:10174000112341F0053008F0ABCE8C2F8F710E9431
:10175000DF10A6CE063008F0A3CEF7CF8C2F8F7106
:10176000112339F00E9499109BCE8C2F8F71112379
:10177000C9F30E94BA1094CE112329F08C2F8F71D7
:101780000E9484108DCE0E947A108ACE112349F0D7
:10179000CF718C2F0E94991063E08C2F0E9427122A
:1017A0007FCE81E00E943012023008F479CE82E0D0
:1017B0000E94301275CE112329F0011159CE8C2FC1
:1017C0008F71D0CF0111CDCE8C2F8F71D2CF4C2FF6
:1017D0004F706D2FC7010E94B5020E94A30F60CE0B
:1017E0004C2F4F706D2FC7010E94140459CEDF910A
:1017F000CF911F910F91FF90EF90DF90BF90AF902E
:101800009F908F9008950F931F93CF93DF93EC01D8
:10181000988189812B813C81232B39F08F3F19F4EA
:1018200081E09F3F19F080E001C081E080FD17C09A
:10183000CE010E94CE02882391F0688179818A814D
:101840000E94F9118C010E9454110E941B10B801D2
:10185000CE01DF91CF911F910F910C94E009DF91A0
:10186000CF911F910F9108950E94EB120E94FC12DC
:101870000E94BE120E9415130E94E3170E943617A1
:1018800090E080E00E94A30790E080E00C94B9070C
:101890000E94DA120C94340C0E94EF11E92FE295A9
:1018A000EF70E250EE30E0F4F0E0E75AF34F0C94C2
:1018B0001D20670C670C700C700C720C700C700C97
:1018C000700C670C670C770C700C700C770C803FF9
:1018D00019F020F4803E20F481E00895843FE1F384
:1018E00080E00895803EC0F3813FD1F7F5CF93FBB0
:1018F000882780F90895CF93DF9300D000D01F92FE
:10190000CDB7DEB70F900F900F900F900F90DF9133
:10191000CF910895CF93DF9300D000D000D0CDB702
:10192000DEB726960FB6F894DEBF0FBECDBFDF91AF
:10193000CF9108951F93CF93DF93C0915C0116E080
:1019400080915D018C1304C0DF91CF911F910895A8
:10195000D0E01C9FF0011D9FF00D1124E25AFE4FB4
:101960004081518162817381848195810E948A0CBA
:101970002196C770E5CF40918E0150918F01609103
:1019800090017091910180919201909193010C943A
:101990008A0C1F93CF93DF9380919301807FD1F4C2
:1019A000809190018823B1F080915C01D0915D011C
:1019B000B0918E01C0918F0140919101509192019F
:1019C000A1E0BF3F09F0A0E0BA016095709516E074
:1019D000D81304C0DF91CF911F91089521E04115E4
:1019E000510521F02A2FCF3F09F020E090E020FDA3
:1019F00038C0189FF001199FF00D1124E25AFE4FD4
:101A000021812C132EC020812B132BC02281211168
:101A100028C0238134812417350700F1241B350B9E
:101A2000283C3105F0F4209193012F702061209320
:101A3000930126E0289FF001299FF00D1124ED5914
:101A4000FE4F80818F70806180838EE891E00E94DC
:101A5000030CDF91CF911F910C949A0C260F371F26
:101A6000DFCF01968770B4CFAF92BF92CF92DF9253
:101A7000EF92FF920F931F93CF93DF93CDB7DEB713
:101A800061970FB6F894DEBF0FBECDBF8C0185E025
:101A9000F801DE011D9601900D928A95E1F7D801BB
:101AA0004C9111965C9111971296EC9030918E01A9
:101AB00060918F01809191019091920121E00097B6
:101AC00031F06F3F19F421E03F3F09F020E0B22FE1
:101AD000B170BB2E20FD80C1F801C380D480A090DE
:101AE0009001AA2009F427C1C816D906D0F1D60161
:101AF000A81BB90BCD01FF24F394883C910508F095
:101B0000F12C80919301982F907FFF2009F4CAC097
:101B1000911187C0FE2C651329C0341327C0E11032
:101B200025C08F708061809393010E94BB0C8EE86A
:101B300091E00E94030C80919301F80185838F2D21
:101B400061960FB6F894DEBF0FBECDBFDF91CF9187
:101B50001F910F91FF90EF90DF90CF90BF90AF90CB
:101B60000895809590958C0D9D1DC5CF81E0CD2861
:101B700031F05F3F19F481E04F3F09F080E080FDD4
:101B800024C081E08E25F82FF170DF2E80FF3FC04A
:101B900080915C0120915D0136E0821318C04D8771
:101BA0005E878D859E850E94EF11292F22952F70CB
:101BB000223008F1243030F59F7009F1D8011596D4
:101BC0009C91907FE1F4FB2CBACF80E0DCCF90E0D9
:101BD000389FF001399FF00D1124E25AFE4F6181C8
:101BE000561306C06081461303C062816E110FC098
:101BF00001968770D2CF9F7011F0882321F3805E09
:101C0000883008F3C8010E94030CBD2CDCCFEE2005
:101C100009F495CF80919301816080939301F12C19
:101C20008ECF651312C0341310C0E1100EC0F8013E
:101C30008583C8010E94030C86E0F801AEE8B1E09C
:101C400001900D928A95E1F741C04D875E878D85A1
:101C50009E850E944C0C882309F4C8C0EE2009F42C
:101C6000C5C080919301803270F020918E01309137
:101C70008F0138872F831986DB86CA868C87CE0131
:101C800007960E94030C86E0F801AEE8B1E00190EF
:101C90000D928A95E1F70E94C90C0E94BB0CFF24AB
:101CA000F3944DCF911115C07C2DD98AC88A6E2D21
:101CB00089890E947B0C8EE891E00E94030C86E0EB
:101CC000EEE8F1E0DF011D928A95E9F70E94BB0C76
:101CD00036CF651312C0341310C0E1100EC0F801E6
:101CE0008583C8010E94030CEEE8F1E086E0DF0185
:101CF0001D928A95E9F7FA2C22CF4D875E878D8554
:101D00009E850E944C0C882309F470C0EE2009F4D3
:101D10006DC080919301803208F4B5CF20918E017F
:101D200030918F013A8329831B82DD82CC828E839E
:101D3000CE010196A6CFC816D90638F1F601E81BE8
:101D4000F90BCF01F12C883C910508F03DC0FE2C29
:101D5000EE2009F44BC0651326C0341324C08091D3
:101D6000930180FD17C0982F907FA1F0D8011596A0
:101D70008C931597903F09F45CCF982F907F905FDC
:101D80008F70892B15968C9354CF809590958C0DE0
:101D90009D1DD8CF86E0F801AEE8B1E001900D922C
:101DA0008A95E1F7CCCE4D875E878D859E850E9412
:101DB0004C0C811168CF80919301816080939301D5
:101DC000C8010E94030CBBCE7C2DD98AC88A6E2D17
:101DD00089890E947B0C73CFEE2041F04D875E878E
:101DE0008D859E850E944C0C81114DCFC8010E94AB
:101DF000030C55CF1F93CF93DF93CDB7DEB72C974E
:101E00000FB6F894DEBF0FBECDBF4F8358876987EA
:101E10007A878B879C87CE0107960E94340D882392
:101E200009F442C09F8188852A853B85232B39F0A0
:101E30008F3F19F481E09F3F19F080E001C081E0FD
:101E400080FD08C04F81588569857A858B859C8582
:101E50000E948A0C16E080915C0190915D018917C7
:101E600009F467C0819FC0011124825A9E4F0E94CD
:101E7000340D882309F45DC0E0915C011E9FF001E0
:101E80001124E25AFE4F4081518162817381848125
:101E900095810E948A0C80915C0190E00196877088
:101EA000992780935C01D7CF86E0FE013796DE014B
:101EB000119601900D928A95E1F79F8188852A8578
:101EC0003B85232B39F08F3F19F481E09F3F19F0B8
:101ED00080E001C081E080FDBDCF20915D0130E058
:101EE000C90101968770992740915C01481719062E
:101EF00099F096E0929FD001939FB00D1124A25AC1
:101F0000BE4FFE01319601900D929A95E1F78093B4
:101F10005D010E949A0C9ECF0E94480C10925D01B8
:101F200010925C0186E0EEE8F1E0DF011D928A95F7
:101F3000E9F72C960FB6F894DEBF0FBECDBFDF9148
:101F4000CF911F910895EF92FF920F931F93CF931C
:101F5000DF938C01892B81F0F12CEE24E394E801CE
:101F60002196F8018491843770F4843008F05FC0C2
:101F70008130B1F08230A1F1DF91CF911F910F91AB
:101F8000FF90EF900895853709F44CC008F43DC0E8
:101F90009CE7980F903780F78F770E94830949C09C
:101FA0000E5F1F4FFE01849190E2980F983060F40D
:101FB0008770FE2D01C0FF0F8A95EAF78F2F0E94D0
:101FC000EE120E94151302C00E94A7088F2D8150A7
:101FD00030F2EFE9FFE03197F1F700C00000F7CFF2
:101FE0000E5F1F4FFE01849190E2980F983050F4DD
:101FF0008770FE2D01C0FF0F8A95EAF78F2F0E9490
:10200000F412DFCF0E948309E1CF0E5F1F4FFE0164
:10201000C491C150D8F28FE99FE00197F1F700C059
:102020000000F7CF0E5F1F4FFE01F490CFCF0E944C
:10203000A7088E01CBCF08956093A7017093A801E4
:102040008093A9019093AA010C94340C0F931F93D1
:102050000091A7011091A8012091A9013091AA0136
:10206000DC01CB01802B912BA22BB32B8093A701FA
:102070009093A801A093A901B093AA011F910F9179
:102080000C94340C0F931F930091A7011091A80199
:102090002091A9013091AA01DC01CB018023912379
:1020A000A223B3238093A7019093A801A093A90131
:1020B000B093AA011F910F910C94340C0F931F93AE
:1020C0000091A7011091A8012091A9013091AA01C6
:1020D000DC01CB0180279127A227B3278093A7019A
:1020E0009093A801A093A901B093AA011F910F9109
:1020F0000C94340C1092A3011092A4011092A5012B
:102100001092A6010C94340C41E050E060E070E0C5
:1021100004C0440F551F661F771F8A95D2F740935E
:10212000A3015093A4016093A5017093A6010C94A0
:10213000340C41E050E060E070E004C0440F551FF3
:10214000661F771F8A95D2F78091A3019091A40111
:10215000A091A501B091A601842B952BA62BB72B9E
:102160008093A3019093A401A093A501B093A6012D
:102170000C94340C41E050E060E070E004C0440F87
:10218000551F661F771F8A95D2F740955095609529
:1021900070958091A3019091A401A091A501B091A7
:1021A000A60184239523A623B7238093A3019093AC
:1021B000A401A093A501B093A6010C94340C41E0B6
:1021C00050E060E070E004C0440F551F661F771FA9
:1021D0008A95D2F78091A3019091A401A091A501C5
:1021E000B091A60184279527A627B7278093A3013E
:1021F0009093A401A093A501B093A6010C94340C74
:102200000F931F930091A3011091A4012091A501A8
:102210003091A601DC01CB01802B912BA22BB32B9B
:102220008093A3019093A401A093A501B093A6016C
:102230001F910F910C94340C0F931F930091A301E5
:102240001091A4012091A5013091A601DC01CB01E0
:1022500080239123A223B3238093A3019093A4010D
:10226000A093A501B093A6011F910F910C94340C7B
:102270000F931F930091A3011091A4012091A50138
:102280003091A601DC01CB0180279127A227B3273B
:102290008093A3019093A401A093A501B093A601FC
:1022A0001F910F910C94340C0895990F990F890F79
:1022B000982F977071E001C0770F9A95EAF786958D
:1022C0008695869525E0829FC001112450E040E06C
:1022D000A62FB0E0FC01E40FF51FEC56FE4F608125
:1022E0009D01042E02C0369527950A94E2F72170CD
:1022F000219526272723262720834F5F5F4F4530D0
:10230000510541F70895990F990F890F982F9770EC
:1023100086958695869525E0829FA001112470E020
:1023200060E080E0FA01E60FF71FEC56FE4F2081D7
:1023300030E0092E02C0369527950A94E2F7217005
:102340003327062E01C0220F0A94EAF7822B6F5F13
:102350007F4F6530710531F70895BF92CF92DF92BC
:10236000EF92FF920F931F93CF93DF938C01C09056
:10237000A301D090A401E090A501F090A601809166
:10238000A7019091A801A091A901B091AA01C82A22
:10239000D92AEA2AFB2ACFE1D0E0BC2ED701C60118
:1023A0000C2E04C0B695A795979587950A94D2F7F9
:1023B00080FD0EC0219788F7B12C8B2DDF91CF9136
:1023C0001F910F91FF90EF90DF90CF90BF900895F5
:1023D000B8018C2F0E943104019761F3EECFCF93A7
:1023E000DF93EC010E94AD11BE01DF91CF910C94FF
:1023F00031041F93CF93DF93EB0190915B019923FD
:1024000031F0CB01DF91CF911F910C94EF11882314
:1024100079F0CB010E94AD11182F682FCE010E94D8
:102420005511BE01812FDF91CF911F910C94310482
:10243000CB010E948311182FF4CF8091AB018595B9
:102440008595859508958091AB018770089598E0F2
:10245000899F90011124622B6093AB010C94991019
:102460009091AB01809589238093AB01282F277031
:1024700061F4282F082E000C330B9217130629F055
:102480008595859585950C94BA1008959091AB012A
:10249000977081E009F480E00895909112019923EA
:1024A000E1F09091010297FF18C0E82FE695E695BC
:1024B000E695EF3139F12091000130910101E20FF1
:1024C000F32FF11D877021E030E001C0220F8A95C3
:1024D000EAF78181822B8183089520910001309158
:1024E0000101F90132969FEF40E05191851751F0BB
:1024F0009F3F19F4511101C0942F4F5F4E31A9F73E
:102500009F3F09F40895290F311D97FD3A95F90170
:1025100082830895909112019923F1F09091010224
:1025200097FF1AC0E82FE695E695E695EF3129F179
:102530002091000130910101E20FF32FF11D282FAE
:10254000277081E090E001C0880F2A95EAF7809516
:1025500091818923818308952091000130910101A7
:10256000F9013296205E3F4F9191891303C0DF013C
:1025700011971C92E217F307B9F7089581E090E0F4
:10258000E0910001F0910101E80FF91F108201961E
:1025900080329105A9F708959091CF01892B8093FE
:1025A000CF010895982F90958091CF018923809332
:1025B000CF0108951092CF0108959091CE01892BFB
:1025C0008093CE010895982F90958091CE01892314
:1025D0008093CE0108951092CE0108959091CD017F
:1025E000892B8093CD010895982F90958091CD01EE
:1025F00089238093CD0108951092CD010895809391
:10260000AC0108951092AC01089520910001309121
:102610000101F9013196205E3F4F80E091919111C7
:102620008F5FE217F307D1F70895E0910001F09171
:1026300001018091CF018083E0910001F0910101BF
:1026400080819091CE01892B8083E0910001F091EF
:10265000010180819091CD01892B80839091AC0103
:10266000992361F0E0910001F09101018081892BB3
:1026700080830E94051381111092AC0180910001AA
:10268000909101010C948D076DEE7EEF90E080E05B
:102690000E94572060E082E090E00E94452060E0C8
:1026A00083E090E00E94452060E084E090E00E949A
:1026B000452060E085E090E00C94452090E080E0CB
:1026C0000E943F2021E08D3E9E4F09F020E0822FA6
:1026D000089582E090E00C943720682F82E090E02B
:1026E0000C94452083E090E00C943720682F83E021
:1026F00090E00C94452084E090E00C943720682F03
:1027000084E090E00C94452080910702843039F1F8
:102710001092D10188E190E020E40FB6F894A895DA
:10272000809360000FBE2093600080E00E9412043E
:1027300083B7817F846083BF83B7816083BF7894D0
:10274000889583B78E7F83BF0FB6F894A895809144
:102750006000886180936000109260000FBE089551
:1027600008950895CF930E94B0130E94CF060E944F
:10277000B113C0E08C2F0E947507811105C0CF5F97
:10278000C530C1F7CF91089581E0FCCF0E94480C7D
:102790000E9481070C9412041F920F920FB60F92A1
:1027A00011248F939F93AF93BF938091D101811197
:1027B00013C08091FD019091FE01A091FF01B091A5
:1027C00000024196A11DB11D8093FD019093FE0171
:1027D000A093FF01B0930002BF91AF919F918F91A1
:1027E0000F900FBE0F901F90189582E084BD93E06C
:1027F00095BD9AEF97BD80936E0008952FB7F8941A
:102800008091FD019091FE01A091FF01B091000225
:102810002FBF0895CF92DF92EF92FF920F931F93F5
:102820002FB7F8944091FD015091FE016091FF0196
:10283000709100022FBF6A017B01EE24FF248C01FE
:1028400030E020E0C016D106E206F30650F0481B47
:10285000590BCA011F910F91FF90EF90DF90CF901D
:10286000089541505109F3CF1F920F920FB60F9266
:1028700011248F939F93AF93BF938091FD0190910B
:10288000FE01A091FF01B09100020196A11DB11DB2
:102890008093FD019093FE01A093FF01B09300028D
:1028A000BF91AF919F918F910F900FBE0F901F908E
:1028B00018950E94DD1BF8942FEF87EA91E62150CE
:1028C00080409040E1F700C0000087E090EBDC0121
:1028D0008093100290931102A0931202B0931302FE
:1028E00088E19CE00FB6F894A895809360000FBE35
:1028F00090936000FFCFCF92DF92EF92FF920F9301
:102900001F93CF93C0E0E82EF12C8C2F0E94750707
:1029100010E000E0C82ED12CC601002E02C0959513
:1029200087950A94E2F780FD11C00F5F1F4F0430B6
:10293000110591F7CF5FC53041F780E0CF911F912E
:102940000F91FF90EF90DF90CF900895602F7C2F34
:1029500080E00E941504E816F90639F781E0EECF11
:10296000CF93C82F8CE20E947B14882321F08C2FF8
:10297000CF910C947B1480E0CF910895CF930E9467
:102980005E13811102C00E944413C5E608C00E9474
:10299000CF068FE39CE90197F1F700C00000C1501A
:1029A000B1F789E20E94B0148111EFC08AE20E945F
:1029B000B01481110E94441385E00E94B01481116B
:1029C0000E9459140E9469138093D00187E00E94ED
:1029D000B014882371F08BE10E94B014882309F4AD
:1029E000B1C09091D001892F8D7F91FF826080933B
:1029F000D0018091D0010E946D130E947B1390E062
:102A0000909302028093010280EE0E94B01488230A
:102A100041F090910102892F8E7F90FF8160809319
:102A2000010289E30E94B014882341F090910102D1
:102A3000892F8D7F91FF82608093010282EE0E9438
:102A4000B014882341F090910102892F8B7F92FF6F
:102A500084608093010286EE0E94B014882341F0C6
:102A600090910102892F877F93FF886080930102F4
:102A700083EE0E94B014882341F090910102892FC7
:102A80008F7E94FF80618093010285E30E94B014E1
:102A9000882341F090910102892F8F7D95FF8062FC
:102AA0008093010281E30E94B014882341F0909149
:102AB0000102892F8F7B96FF80648093010281E160
:102AC0000E94B014882341F090910102892F97FB56
:102AD00087F9805880930102809101020E947F1340
:102AE00087E20E94B014C82F8EE10E94B0148111B9
:102AF000C2608FE10E94B0148111C46080E20E9424
:102B0000B0148111C86081E20E94B0148111C061CB
:102B100082E20E94B0148111C06283E20E94B0146C
:102B20008111C06484E20E94B014882341F1C0681E
:102B30008C2F0E9476136C2F70E090E080E0CF9194
:102B40000C941C108EE00E94B014882339F09091F0
:102B5000D001892F8B7F92FF846049CF80E10E9452
:102B6000B0149091D001882329F0892F877F93FF9B
:102B700088603DCF892F8E7F90FF816038CFC11153
:102B8000D7CF0E947213682FD7CFCF91089580912D
:102B9000D40180FF12C06091050185E0689FB001FB
:102BA0001124759567957595679560387105A8F539
:102BB00061157105A1F1862F089581FF09C060910B
:102BC000050185E0689FB001112475956795EDCFEB
:102BD00082FF07C06091050185E0689FB001112464
:102BE000E4CF2091D5012223A9F0909104016091B6
:102BF000050185E0689FB00111242917B0F6269FD2
:102C0000A001279F500D1124692F70E0CA010E9476
:102C10000920CBCF65E070E0CECF8FE7089581E04B
:102C200008958091D40180FF0CC06091030170E091
:102C300075956795759567956115710549F1862FAD
:102C4000089581FF06C06091030170E07595679556
:102C5000F3CF6091030182FD0BC09091D5019923C0
:102C6000A1F06091020180910301961738F0682F5E
:102C700070E06038710500F38FE70895899FC00107
:102C8000112470E00E940920F4CF61E070E0D7CFFA
:102C900081E00895803F31F40E94C71581958093AB
:102CA000D8010895813F19F40E94C715F8CF823FDB
:102CB00031F40E94C71581958093D7010895833F11
:102CC00019F40E94C715F8CF893F29F40E94111604
:102CD0008093D90108958A3F21F40E9411168195AD
:102CE000F7CF8B3F31F40E94111681958093DA0162
:102CF00008958C3F19F40E941116F8CF843F31F4E7
:102D00008091D60181608093D6010895853F21F49A
:102D10008091D6018260F7CF863F21F48091D60161
:102D20008460F1CF873F21F48091D6018860EBCF9A
:102D3000883F21F48091D6018061E5CF8D3F31F449
:102D40008091D40181608093D40108958E3F21F455
:102D50008091D4018260F7CF8F3FB9F78091D40181
:102D60008460F1CF803FC1F48091D80187FD10923B
:102D7000D8018091D70181110EC08091D8018111B5
:102D80000AC08091D901811106C08091DA018111B8
:102D900002C01092D5010895813F29F48091D80195
:102DA00018162CF3E6CF9091D701823F29F497FFB4
:102DB000E0CF1092D701DDCF833F19F41916CCF381
:102DC000D8CF893F39F48091D901181694F6109222
:102DD000D901CFCF8A3F29F48091D90187FFC9CF8C
:102DE000F6CF8B3F39F48091DA0187FFC2CF109282
:102DF000DA01BFCF8C3F29F48091DA011816BCF3B9
:102E0000B8CF843F31F48091D6018E7F8093D60174
:102E1000B0CF853F21F48091D6018D7FF7CF863FDB
:102E200021F48091D6018B7FF1CF873F21F48091EF
:102E3000D601877FEBCF883F21F48091D6018F7E2A
:102E4000E5CF8D3F31F48091D4018E7F8093D40102
:102E500090CF8E3F21F48091D4018D7FF7CF8F3FAB
:102E600009F087CF8091D4018B7FF0CF86ED91E080
:102E70000E9498070E94FE139093D3018093D20181
:102E800008951F93CF93DF938091D2019091D30146
:102E90000E940A14AC019091D5012091060130E006
:102EA000911106C0209107018AE0289F900111240A
:102EB0004217530780F08091D701C091D80110913B
:102EC000D901D091DA0181110AC0C11178C0111164
:102ED00076C0D11174C0DF91CF911F9108959F3FAB
:102EE00019F09F5F9093D501181624F40E94C7151E
:102EF0008093D7018091D70187FF05C00E94C71535
:102F000081958093D7011C1624F40E94C7158093E5
:102F1000D8018091D80187FF05C00E94C71581950F
:102F20008093D8016091D701662331F1C091D80117
:102F3000CC2311F1062E000C770B880B990B0E9405
:102F4000101F23E333E343E35FE30E94741F0E94F7
:102F5000D81E6093D7016C2FCC0F770B880B990B81
:102F60000E94101F23E333E343E35FE30E94741FD7
:102F70000E94D81E6093D801111624F40E941116E5
:102F80008093D9018091D90187FF05C00E94111655
:102F900081958093D9011D1624F40E941116809307
:102FA000DA018091DA0187FF05C00E941116819530
:102FB0008093DA01DF91CF911F910C9436179F3FD8
:102FC00009F08FCFA0CF85E0E6EDF1E0DF011D92A3
:102FD0008A95E9F71092D5011092D4010895809155
:102FE000FB010895CF93DF9300D01F92CDB7DEB7DA
:102FF0009C0180910702843019F593E099833B830B
:103000002A839093E9008FEF9091E800815095FD1D
:1030100006C095ED9A95F1F700008111F5CF8091EA
:10302000E80085FF0DC050E040E063E070E0CE01B5
:1030300001960E944D1A8091E8008E778093E800F7
:103040000F900F900F90DF91CF910895CF93DF9362
:1030500000D01F92CDB7DEB720910702243031F5A2
:1030600022E02983805891099B838A8383E080939F
:10307000E9008FEF9091E800815095FD06C095ED35
:103080009A95F1F700008111F5CF8091E80085FF56
:103090000DC050E040E063E070E0CE0101960E9478
:1030A0004D1A8091E8008E778093E8000F900F9082
:1030B0000F90DF91CF9108959C0180910702843099
:1030C000F9F482E08093E9009FEF8091E80091504D
:1030D00085FD06C085ED8A95F1F700009111F5CFC9
:1030E0008091E80085FF0CC050E040E065E070E0B2
:1030F000C9010E944D1A8091E8008E778093E80004
:103100000895CF93DF93EC01809107028430F1F4AE
:10311000909112019923E9F09091010297FF19C053
:103120008093E9008FEF9091E800815095FD06C0F3
:1031300095E19A95F1F700008111F5CF8091E800B3
:1031400050E040E060E270E085FD1AC0DF91CF9171
:10315000089581E08093E9008FEF9091E80081501D
:1031600095FD06C095ED9A95F1F700008111F5CF18
:103170008091E80085FFEACF50E040E068E070E031
:10318000CE010E944D1A8091E8008E778093E8006E
:1031900080E2FE01ABEDB1E001900D928A95E1F77E
:1031A000D5CF80910602811109C00E94DD1B0E94CB
:1031B0003A1C8091E20084608093E20008951092AE
:1031C00006020895089508950C94C61342E061EC38
:1031D00081E00E945B1B42E061EC82E00E945B1B8D
:1031E00042E061EC83E00E945B1B42E261EC84E020
:1031F0000C945B1B80910902833009F455C030F4B4
:10320000813071F1823009F491C008958A3009F457
:103210007DC08B3009F463C0893009F044C08091CF
:103220000802813209F03FC080910C0290910D029A
:10323000009711F00397B9F58091E800877F80939C
:10324000E8008091E80082FF2AC08091F10080931D
:10325000FB018091E8008B778093E8000C948F1B32
:1032600080910802813AF9F48091E800877F809389
:10327000E80080910C0290910D02892B61F460E2CC
:103280008BED91E070E00E949C1A8091E8008B77B2
:103290008093E800089560E090E080E0F3CF8091B3
:1032A00007028111CECF089580910802813AD9F7A3
:1032B00080910C0290910D02892BA9F78091E80072
:1032C000877F8093E8008091E80080FFFCCF8091A9
:1032D00012018093F1008091E8008E77BDCF80913C
:1032E0000802813201F780910C0290910D02892B26
:1032F000D1F68091E800877F8093E8000E948F1BC1
:1033000080910A02809312010C94480C809108026B
:10331000813249F68091E800877F8093E8000E941F
:103320008F1B80910B028093FC010895809108020D
:10333000813A09F0B8CF8091E800877F8093E80058
:103340008091E80080FFFCCF8091FC01C2CF84B760
:10335000877F84BF0FB6F894A8958091600088613C
:1033600080936000109260000FBE80E8809361003F
:10337000109261000E94D0070E94DD1B0E943A1C3F
:103380008091E20084608093E20078940E94BC1EE9
:103390000E94D20788E091E00E947C07809107029A
:1033A000853019F00E94D807F9CF0E9484138091CC
:1033B0000502882399F30E94B213882379F30E94AF
:1033C000371AECCF292F33272330310579F158F400
:1033D00021303105F1F02230310519F190E080E023
:1033E00030E020E01AC02132310599F12232310556
:1033F000A9F7643098F770E0FB01EE0FFF1FE05E65
:10340000FE4F20813181645E7E4FFB01808190E020
:1034100004C082E190E029EC33E0FA01318320839B
:1034200008958DE690E02CE533E0F7CF99278130C1
:10343000910561F028F0029789F6ECE2F3E002C012
:10344000E8E5F3E0849190E09F01E7CFE0E4F3E06A
:10345000F9CF643008F0C2CFE62FF0E0EE0FFF1F87
:10346000E85DFE4F2081318189E090E0D6CF80E198
:1034700089BD82E189BD09B400FEFDCF8091D800ED
:103480008F7D8093D8008091E00082608093E0007F
:103490008091E00081FDFCCF0895AF92BF92CF9262
:1034A000DF92FF920F931F93CF93DF936C01EB0199
:1034B0008A010E94AE1BF82E811123C0011511054F
:1034C00039F0F80180819181C81BD90BC80ED91E33
:1034D000B12CA12C2097A9F08091E80085FD22C095
:1034E0008091E8008E778093E80001151105A1F026
:1034F000F80180819181A80EB91EB182A08285E079
:10350000F82E8F2DDF91CF911F910F91FF90DF90BB
:10351000CF90BF90AF9008950E94AE1B8823D1F248
:10352000F82EEFCFF60181916F018093F100219782
:10353000FFEFAF1ABF0ACECFFC0180910E0290912F
:103540000F0286179707A0F06115710529F4909175
:10355000E8009E779093E80090E06115710551F4C2
:10356000911108C08091E80082FF35C080E0089585
:10357000BC01F2CF809107028823C9F18530C9F1DF
:103580008091E80083FD31C08091E80082FDEACFA0
:103590008091E80080FFE1CF2091F3008091F2005C
:1035A000322F282F6115710519F02830310558F098
:1035B00091E02830310509F090E02091E8002E7765
:1035C0002093E800CACF81918093F1006150710986
:1035D0002F5F3F4FE7CF80910702882341F085306E
:1035E00041F08091E80083FFBDCF81E0089582E043
:1035F000089583E00895FC0180910E0290910F02DE
:1036000086179707A0F06115710529F48091E800ED
:103610008E778093E80090E06115710551F4911167
:1036200008C08091E80082FF36C080E00895BC01A8
:10363000F2CF809107028823D1F18530D1F18091BA
:10364000E80083FD32C08091E80082FDEACF8091DE
:10365000E80080FFE1CF2091F3008091F200322F4B
:10366000282F6115710519F02830310558F091E0C7
:103670002830310509F090E08091E8008E77809342
:10368000E800CACF84918093F100319661507109AE
:103690002F5F3F4FE6CF80910702882341F08530AE
:1036A00041F08091E80083FFBCCF81E0089582E083
:1036B000089583E00895982F973028F08F708093B5
:1036C000E90081E008959093E900242F762F50E0DF
:1036D000981731F07091EC002091ED005091F000BE
:1036E00021FD02C09F5FE8CF3091EB003E7F309319
:1036F000EB003091ED003D7F3093ED003091EB0019
:1037000031603093EB007093EC002093ED00509308
:10371000F0002091EE0027FDE5CF80E00895809134
:10372000080287FF13C08091E80082FF06C08091E5
:10373000E8008B778093E80004C080910702811134
:10374000F2CF0895809107028823D9F38091E80091
:1037500080FFF8CF8091E8008E77ECCF2091E400D5
:103760003091E50085E69091EC0090FF06C09091C5
:10377000E80090FF06C080E008959091E80092FD77
:10378000FACF90910702992391F0953091F09091A2
:10379000EB0095FD10C04091E4005091E500241726
:1037A000350709F381509A01F1F684E0089582E02B
:1037B000089583E0089581E008950E944B1C0E94C3
:1037C000531CE0EEF0E0808181608083E8EDF0E062
:1037D00080818F77808319BCA7EDB0E08C918E7FBC
:1037E0008C9380818F7E80831092060208950F93C0
:1037F0001F93CF93DF930E944B1C0E94531CC8ED74
:10380000D0E088818F7788838881806888838881E9
:103810008F7D888319BC10920702109203021092C8
:1038200005021092040200EE10E0F80180818B7F07
:10383000808388818160888342E060E080E00E942C
:103840005B1BE1EEF0E080818E7F8083E2EEF0E0B2
:10385000808181608083808188608083F80180819D
:103860008E7F8083888180618883DF91CF911F91D3
:103870000F910895E8EDF0E080818F7E8083E7ED81
:10388000F0E080818160808384E082BF81E080936A
:1038900006020C94F71BE8EDF0E080818E7F8083B8
:1038A0001092E20008951092DA001092E10008955B
:1038B0001F920F920FB60F9211242F933F934F93A5
:1038C0005F936F937F938F939F93AF93BF93EF9388
:1038D000FF938091E10082FF0BC08091E20082FFA4
:1038E00007C08091E1008B7F8093E1000E94BB1EA6
:1038F0008091DA0080FF19C08091D80080FF15C048
:103900008091DA008E7F8093DA008091D90080FF69
:1039100094C080E189BD82E189BD09B400FEFDCF7C
:1039200081E0809307020E94D1188091E10080FF1E
:1039300019C08091E20080FF15C08091E2008E7F67
:103940008093E2008091E20080618093E2008091A8
:10395000D80080628093D80019BC85E0809307026C
:103960000E94E3188091E10084FF29C08091E20069
:1039700084FF25C080E189BD82E189BD09B400FED4
:10398000FDCF8091D8008F7D8093D8008091E10099
:103990008F7E8093E1008091E2008F7E8093E20031
:1039A0008091E20081608093E2008091030288238D
:1039B00009F449C084E0809307020E94E4188091D2
:1039C000E10083FF29C08091E20083FF25C0809140
:1039D000E100877F8093E10082E0809307021092EC
:1039E00003028091E1008E7F8093E1008091E200EC
:1039F0008E7F8093E2008091E20080618093E200FC
:103A000042E060E080E00E945B1B8091F0008860F3
:103A10008093F0000E94E218FF91EF91BF91AF9167
:103A20009F918F917F916F915F914F913F912F91D6
:103A30000F900FBE0F901F90189519BC109207029F
:103A40000E94DF1872CF8091E30087FD02C081E001
:103A5000B2CF83E0B0CF1F920F920FB60F92112416
:103A60002F933F934F935F936F937F938F939F9386
:103A7000AF93BF93CF93EF93FF93C091E900CF70C3
:103A80008091EC001092E9008091F000877F809394
:103A9000F00078940E94671D1092E9008091F00078
:103AA00088608093F000C093E900FF91EF91CF917F
:103AB000BF91AF919F918F917F916F915F914F9146
:103AC0003F912F910F900FBE0F901F9018951F934D
:103AD000CF93DF93CDB7DEB7AA970FB6F894DEBFCA
:103AE0000FBECDBFE8E0F2E08091F100819322E0CB
:103AF000E031F207C9F70E94FA188091E80083FFCD
:103B000042C080910802909109029A3008F03BC0AF
:103B1000E92FF0E0E257F24E0C941D20981DBC1DD9
:103B2000C31DBC1DC31D171E391EC31D8E1E9B1E2B
:103B3000803879F0823839F580910C028F7080934B
:103B4000E9008091EB0085FB882780F91092E9005D
:103B500006C08091040290910502911182609091BB
:103B6000E800977F9093E8008093F1001092F100B5
:103B70008091E8008E772DC0282F2D7F21F4882397
:103B8000D1F0823059F18091E80083FF0AC0809122
:103B9000E800877F8093E8008091EB00806280934B
:103BA000EB00AA960FB6F894DEBF0FBECDBFDF9133
:103BB000CF911F91089580910A02813021F79330AF
:103BC00009F080E0809305021092E9008091E800FE
:103BD000877F8093E8000E948F1BD5CF80910A02D7
:103BE0008111F2CF80910C028F7069F28093E9000D
:103BF0002091EB0020FFE8CF933031F48091EB006F
:103C000080628093EB00E0CF9091EB009061909305
:103C1000EB0021E030E001C0220F8A95EAF7209303
:103C2000EA001092EA008091EB008860EACF8111EF
:103C3000AACF10910A021F778091E3008078812B30
:103C40008093E3008091E800877F8093E8000E94E2
:103C50008F1B8091E80080FFFCCF8091E30080689B
:103C60008093E30083E0111101C082E0809307029A
:103C70008ACF8058823008F086CF80910A029091D6
:103C80000B028C3D23E09207A1F583E08A838AE250
:103C900089834FB7F894DE01139620E03EE051E2AD
:103CA000E32FF0E050935700E49120FF03C0E2952A
:103CB000EF703F5FEF708E2F90E0EA30C0F0C79654
:103CC0008D939D932F5F243159F74FBF8091E8006A
:103CD000877F8093E8006AE270E0CE0101960E943F
:103CE0009C1A8091E8008B778093E8004CCFC096B7
:103CF000E7CFAE014F5F5F4F60910C020E94E21967
:103D0000BC01892B09F43FCF9091E800977F9093F5
:103D1000E80089819A810E94FB1AE3CF803809F07C
:103D200032CF8091E800877F8093E8008091030282
:103D30008093F1001DCF811126CF90910A0292301D
:103D400008F021CF8091E800877F8093E80090936E
:103D500003020E948F1B80910302882331F084E0CC
:103D6000809307020E94E6180ECF8091E30087FD42
:103D7000F6CF81E0F5CF0895CF9380910702882395
:103D800099F0C091E900CF708091EC0080FD0EC0E9
:103D900080E0C82B1092E9008091E80083FD0E942A
:103DA000671DCF70C093E900CF91089580E8F1CFEF
:103DB0000E94DF1E6894B1110C946E1F08950E943A
:103DC000531F88F09F5798F0B92F9927B751B0F03B
:103DD000E1F0660F771F881F991F1AF0BA95C9F78F
:103DE00014C0B13091F00E946D1FB1E008950C94A1
:103DF0006D1F672F782F8827B85F39F0B93FCCF354
:103E0000869577956795B395D9F73EF4909580950B
:103E1000709561957F4F8F4F9F4F0895E89409C02B
:103E200097FB3EF490958095709561957F4F8F4FED
:103E30009F4F9923A9F0F92F96E9BB279395F69503
:103E4000879577956795B795F111F8CFFAF4BB0F81
:103E500011F460FF1BC06F5F7F4F8F4F9F4F16C0E5
:103E6000882311F096E911C0772321F09EE8872F6F
:103E7000762F05C0662371F096E8862F70E060E02B
:103E80002AF09A95660F771F881FDAF7880F9695A4
:103E9000879597F9089557FD9058440F551F59F08D
:103EA0005F3F71F04795880F97FB991F61F09F3F27
:103EB00079F087950895121613061406551FF2CF50
:103EC0004695F1DF08C0161617061806991FF1CFA0
:103ED00086957105610508940895E894BB276627C7
:103EE0007727CB0197F908950E94871F0C94F81F3C
:103EF0000E94EA1F38F00E94F11F20F0952311F074
:103F00000C94E11F0C94E71F11240C946E1F0E9467
:103F10004B1F70F3959FC1F3950F50E0551F629FA3
:103F2000F001729FBB27F00DB11D639FAA27F00D12
:103F3000B11DAA1F649F6627B00DA11D661F829F39
:103F40002227B00DA11D621F739FB00DA11D621F1E
:103F5000839FA00D611D221F749F3327A00D611D3B
:103F6000231F849F600D211D822F762F6A2F11241D
:103F70009F5750409AF0F1F088234AF0EE0FFF1F50
:103F8000BB1F661F771F881F91505040A9F79E3FA7
:103F9000510580F00C94E11F0C946E1F5F3FE4F319
:103FA000983ED4F3869577956795B795F795E795FD
:103FB0009F5FC1F7FE2B880F911D9695879597F906
:103FC000089597F99F6780E870E060E008959FEF9B
:103FD00080EC089500240A941616170618060906A0
:103FE000089500240A94121613061406050608956F
:103FF000092E0394000C11F4882352F0BB0F40F4F7
:10400000BF2B11F460FF04C06F5F7F4F8F4F9F4F36
:10401000089597FB072E16F4009407D077FD09D07A
:104020000E94232007FC05D03EF4909581959F4F78
:104030000895709561957F4F0895EE0FFF1F0590CD
:10404000F491E02D0994AA1BBB1B51E107C0AA1FE4
:10405000BB1FA617B70710F0A61BB70B881F991F29
:104060005A95A9F780959095BC01CD010895F999CD
:10407000FECF92BD81BDF89A992780B50895A8E139
:10408000B0E042E050E00C945F20262FF999FECF7B
:1040900092BD81BDF89A019700B4021639F01FBA9B
:1040A00020BD0FB6F894FA9AF99A0FBE08950196BA
:1040B000272F0E9446200C944520DC01CB01FC01F7
:1040C000F999FECF06C0F2BDE1BDF89A319600B471
:0E40D0000D9241505040B8F70895F894FFCF7C
:1040DE00AD012808140A321EEF1781185C18261835
:1040EE00F21701F4F5F6F7946697C634404D36395B
:1040FE0097044A041404DB036E038703A003B90379
:00000001FF
